:020000006E2F61
:08000800FF00030E8312031335
:10001000B4000A0EB500040EB6008A110A12A92F08
:10002000D208031D14280800F5300000000000006D
:1000300000000000000000000000000000000000C0
:1000400000000000000000000000FF3E031D152816
:1000500000000000000000000000000000000000A0
:1000600000000000000000000000D20B142808006F
:100070007308F700F6010310F70DF60DF70DF60DF6
:10008000F7070318F60AF7070318F60A5130F707BF
:100090000318F60A003076078A007408F60077081D
:1000A000820000308A000030F70085307E28003062
:1000B0008A000030F700C1307E2800308A0000300E
:1000C000F700FD307E2800308A000130F70039301B
:1000D0007E2800308A000130F70075307E2800301D
:1000E0008A000130F700B1307E2800308A000130EC
:1000F000F700ED307E280230F7002930F6070318AC
:10010000F70A77088A007608820000340034003449
:1001100000340034003406345F34063400340734CD
:10012000033400340734033424347E3424347E34DE
:10013000243424342B346A341234003463341334BA
:1001400008346434633436344934563420345034FB
:100150000034073403340034003400343E34413476
:1001600000340034003441343E3400340034083468
:100170003E341C343E340834083408343E340834E9
:1001800008340034E0346034003400340834083477
:1001900008340834083400346034603400340034E7
:1001A000203410340834043402343E345134493499
:1001B00045343E34003442347F34403400346234B9
:1001C0005134493449344634223449344934493469
:1001D00036341834143412347F3410342F34493404
:1001E0004934493431343C344A3449344934303464
:1001F0000134713409340534033436344934493414
:100200004934363406344934493429341E340034F0
:100210006C346C34003400340034EC346C3400340E
:100220000034083414342234413400342434243467
:100230002434243424340034413422341434083433
:10024000023401345934093406343E3441345D34C7
:1002500055341E347E340934093409347E347F34F5
:1002600049344934493436343E34413441344134DC
:1002700022347F344134413441343E347F34493474
:100280004934493441347F34093409340934013460
:100290003E344134493449347A347F3408340834A4
:1002A00008347F34003441347F34413400343034F6
:1002B0004034403440343F347F34083414342234E2
:1002C00041347F3440344034403440347F3402344D
:1002D000043402347F347F340234043408347F34ED
:1002E0003E344134413441343E347F34093409349E
:1002F000093406343E344134513421345E347F3481
:1003000009340934193466342634493449344934BB
:100310003234013401347F34013401343F34403409
:10032000403440343F341F342034403420341F34B0
:100330003F3440343C3440343F3463341434083464
:100340001434633407340834703408340734713497
:10035000493445344334003400347F34413441342B
:10036000003402340434083410342034003441346E
:1003700041347F3400340434023401340234043410
:100380008034803480348034803400340334073443
:1003900000340034203454345434543478347F34AA
:1003A00044344434443438343834443444344434A5
:1003B000283438344434443444347F343834543466
:1003C00054345434183408347E3409340934003435
:1003D0001834A434A434A4347C347F340434043476
:1003E00078340034003400347D3400340034403438
:1003F000803484347D3400347F34103428344434E1
:100400000034003400347F34403400347C3404340D
:100410001834043478347C340434043478340034AC
:1004200038344434443444343834FC34443444346C
:10043000443438343834443444344434FC3444345C
:100440007834443404340834083454345434543440
:10045000203404343E344434243400343C344034B6
:1004600020347C3400341C342034403420341C3498
:100470003C346034303460343C346C3410341034E8
:100480006C3400349C34A03460343C340034643424
:10049000543454344C34003408343E344134413400
:1004A0000034003400347F340034003400344134EC
:1004B00041343E340834023401340234013400340F
:1004C000FB08031D6D2A8312031387151030831652
:1004D000A000A1018030A200762A831203138711A5
:1004E00008308316A0008030A100A20183120711FA
:1004F000FE01831620087E020318962A83128710B5
:10050000831621087C05031D892A22087D0503190D
:100510008C2A831207148E2A831207108714FC0872
:10052000FD080310FC0DFD0DFE0A792A8312071544
:100530000800F701FA01FB017308F800F901F71947
:100540000800741CA92A7808FA070318FB0A79081E
:10055000FB07F40C0310F80DF90DF70A9F2AFB01B5
:100560009030FC00EF30FD006022FB01FC01053003
:10057000FD006022FB0177080038FC000830FD0018
:100580006022FB0179080038FC000930FD00602280
:10059000FB0178080038FC000A30FD006022FB01F6
:1005A0007A080038FC000B30FD0060220800F501DD
:1005B000831374188317730884007508F50A840779
:1005C0008008031DD82AF5030800E601E901EA01C5
:1005D0006208E7006308E800E51FF42AE617E4096B
:1005E000E509E40A0319E50A661A062B641CFE2ACB
:1005F0006708E90768080318680FEA070310E50CA5
:10060000E40C0310E70DE80DE60AF42AE61F0800E3
:10061000E909EA09E90A0319EA0A0800750AF50076
:10062000760AF6007508F7007608F8007508F900F4
:100630007608FA00AF220130FB005008FC00FD01F3
:1006400060220800843083120313D200B030D3003C
:10065000F701F8015203F9005303FA00AF225208E0
:10066000F3005308F40099227A08D4007B08D500DF
:10067000D601D7015708803AD8005508803A580269
:10068000031D442B54085602031808000130FB00D8
:100690005108FC00FD016022D60A0319D70A3A2B43
:1006A0005208073C0318562B0730D2005308073C6A
:1006B00003185C2B0730D3005408033C0318622B4B
:1006C0000330D400D308D30DD30DFC30D305D208AA
:1006D000D20DD20DD20DD20DD20DE030D20552087E
:1006E0005404D1005308D10408005308073C0318F0
:1006F0007B2B0730D3005408073C0318812B0730AD
:10070000D4005508033C0318872B0330D500D408C8
:10071000D40DD40DFC30D405D308D30DD30DD30D97
:10072000D30DD30DE030D30553085504D000540841
:10073000D0040800DA01DB01DD0152085402DC00BC
:10074000031CDD03DF0153085502DE00031CDF0339
:100750000130E000E100DD1FBC2BFF30E0005C0851
:10076000E2005D08E300FF30E400E501E503E52277
:100770006908DC006A08DD00DF1FCD2BFF30E100D7
:100780005E08E2005F08E300FF30E400E501E503F6
:10079000E5226908DE006A08DF005D08803AE200B1
:1007A0005F08803A6202031DD72B5E085C02031CBF
:1007B000132C5C08D6005D08D7000310D60DD70DAA
:1007C0005E08D8005F08D9000310D80DD90D540871
:1007D0005206031908005208F5005308F6000E23CC
:1007E00060085207D2005808DA075908E2005B088F
:1007F0000318E20AE2076208DB005D08803AE200C3
:100800005B08803A6202031D072C5A085C02031839
:10081000E72B61085307D3005608DA02570A03187A
:100820005708DB02E72B5E08E2005F08E3000310D5
:10083000E20DE30D6208D6006308D7005C08E20011
:100840005D08E3000310E20DE30D6208D8006308C1
:10085000D900550853060319552C5208F5005308C2
:10086000F6000E2361085307D3005808DA07590829
:10087000E2005B080318E20AE2076208DB005F0897
:10088000803AE2005B08803A6202031D492C5A0854
:100890005E020318292C60085207D2005608DA02BB
:1008A000570A03185708DB02292C5208F500530891
:1008B000F6000E2308000130EA00EB00F2015208B6
:1008C000F3005308F400D7227508E3005E03031D0C
:1008D0006B2C0230EA005E08023A031D722C0230D3
:1008E000EA00EB005E08033A031D782C0230EB00AF
:1008F000E501E90163086902031808006908520765
:10090000F3005308F4000318F40A831374188317D0
:100910007308840020300002E200E4010530640224
:100920000318992D0C3062020318B12C6208F300F1
:100930000530F40099227A08EC007B08F500640881
:10094000EC074808F3006C08F4003820F500831326
:100950006D30840064088407750880008A110A12CB
:10096000952D183062020318D22C0C306202F3006D
:100970000530F40099227A08F5007B08F600640837
:100980007507EC004908F3006C08F4003820F50006
:1009900083136D30840064088407750880008A1111
:1009A0000A12952D243062020318F32C18306202CB
:1009B000F3000530F40099227A08F5007B08F60070
:1009C00064087507EC004A08F3006C08F40038204E
:1009D000F50083136D308400640884077508800077
:1009E0008A110A12952D303062020318142D24301A
:1009F0006202F3000530F40099227A08F5007B08C2
:100A0000F60064087507EC004B08F3006C08F4006E
:100A10003820F50083136D3084006408840775085E
:100A200080008A110A12952D3C3062020318352D80
:100A300030306202F3000530F40099227A08F500A4
:100A40007B08F60064087507EC004C08F3006C089E
:100A5000F4003820F50083136D30840064088407A7
:100A6000750880008A110A12952D48306202031819
:100A7000562D3C306202F3000530F40099227A08CA
:100A8000F5007B08F60064087507EC004D08F300DC
:100A90006C08F4003820F50083136D30840064087E
:100AA0008407750880008A110A12952D543062025D
:100AB0000318772D48306202F3000530F4009922C4
:100AC0007A08F5007B08F60064087507EC004E080C
:100AD000F3006C08F4003820F50083136D308400B7
:100AE00064088407750880008A110A12952D5F300A
:100AF00062020318952D54306202F3000530F400B1
:100B000099227A08F5007B08F60064087507EC0066
:100B10004F08F3006C08F4003820F50083136D30A3
:100B200084006408840775088000E40A8A110A12A8
:100B30008E2CE001063060020318FB2DE8016A08E4
:100B400068020318F92DE601E1010830610203187B
:100B5000F62DE7016B0867020318F42D83136D303F
:100B60008400600884070130F300F4016108FF3954
:100B70000319BF2D0310F30DF40DFF3EB72D7308BD
:100B800000050319CB2D65085C07F50066085D07B5
:100B9000F6000E23F12DDF08031DF12DF501650888
:100BA0005C07F7000318F50AF70AF50166085D0708
:100BB000F8000318F50AF80AF50165085C07F90062
:100BC0000318F50AF90AF50166085D07FA0003182B
:100BD000F50AFA0AAF220130FB005108FC00FD01C2
:100BE0006022E60AE70AAA2DE10AA52DE50AE80A2D
:100BF0009F2DE00A9A2DE90A7A2C83160313871198
:100C00000711071087100A308312D20010208714B2
:100C10008715071507140A30D2001020FB01FD309C
:100C2000FC00FD006022FB01FD30FC00FD006022A5
:100C3000FB01FC01EF30FD006022FB010430FC00F1
:100C4000EE30FD006022FB010430FC001B30FD0093
:100C50006022FB01FE30FC00FD006022FB01FE3043
:100C6000FC00FD006022FB019030FC00EF30FD0035
:100C70006022FB010430FC004A30FD006022FB01D1
:100C80003F30FC007F30FD006022FB010430FC009F
:100C9000EE30FD006022FB010630FC004330FD0019
:100CA00060220730D2001020FB019030FC00EF30B2
:100CB000FD006022FB018330FC000930FD00602252
:100CC000FB01FC010830FD006022FB01AF30FC009D
:100CD0000B30FD006022FB01FC010A30FD006022A8
:100CE000FB01FC010530FD006022FB01FC01063028
:100CF000FD006022FB01FC010730FD006022FB01CA
:100D0000FC01EF30FD006022FB010C30FC00EE30F6
:100D1000FD006022FB019030FC00EF30FD006022FE
:100D2000FB018030FC00FD016022FB01B030FC00C3
:100D3000EF30FD006022FB010230FC004930FD0075
:100D40006022FB01FC01EF30FD006022FB0101305D
:100D5000FC007F30FD006022FB018130FC00E130AF
:100D6000FD006022FB010230FC00E230FD00602249
:100D7000FB017630FC00E230FD006022FB01833095
:100D8000FC00E130FD006022FB010130FC008030FE
:100D9000FD006022FB019030FC00EF30FD0060227E
:100DA000FB01FC01FD016022FB019030FC00EF30F3
:100DB000FD006022FB010130FC00E830FD006022F4
:100DC000222308000730831603139F00C0308100E0
:100DD000FD2522234630D200D3005A30D4004630BD
:100DE000D5009A235030D2003C30D3005030D4008C
:100DF000D5009A230730D300D401D501752346309E
:100E0000D2005030D3005A30D4003C30D5009A2361
:100E1000D301D4010330D50075234630D2003C30D5
:100E2000D3005A30D4005030D5009A23D301D401D6
:100E3000D50175230730D2000530D300D4015023EB
:100E40004D30D4006130D5007430D6007230D700F8
:100E50006930D8007830D900DA010030D30054303E
:100E6000D2000630DB000A30DC006E30DD000130DD
:100E7000DE00DF015B24C5010F304505C2004830AC
:100E8000C207450E0F39C3001430C30703304505B0
:100E9000C400450CC700C70C3F30C7050730C70565
:100EA000450CC600C60E0730C6050730C605460805
:100EB000D3004708D4004408D50075234208F50044
:100EC0004308F6000E23450AC500D201D20AC50820
:100ED000031D5210D20803193C2F6D2FD5308312F9
:100EE0000313A000C430A100BB30A200DC30A3007B
:100EF000A401A501A601A701A801A901AA01AB01AE
:100F0000AC01AD01AE01AF01BC01BD01B701B8013B
:100F1000BE01BF01C001C101B001B101B201B30105
:100F2000BA01BB01B9010030C8000130C90002306C
:100F3000CA000330CB000430CC000530CD000630B1
:100F4000CE000730CF00D001FF30D1008A110A1245
:100F5000E22E83120313360E8400350E8A00340EFF
:080F60008300FF0E7F0E090063
:00000001FF
